:020000040000FA
:0600000000000EEF00F00D
:0400080004EF00F011
:080018000CEF00F00BD8817021
:1000200055D991D8E1D87BD8E6D8B6D8F8D81DD91B
:1000300054D9F5D74E0EC16E610EC26EE10E926EAE
:10004000DC0E936ED20E946E0F0E956E040E966EAD
:10005000100E806E200EC66EC00EC76E080EB16EFA
:10006000810ECD6E0B0EBD6E610EBF6EA80EBE6E04
:1000700083CF03F0156A080E046E056A066AC00E87
:10008000096EDF0E0C6E460E0D6E000E0E6E000E2B
:10009000126E06D8020EF76EEA0EF66E1FD8120028
:1000A0000A0E006E1AD90006FDE18490020EF76E6A
:1000B000E20EF66E08008482F5CF83FF84920DD99C
:1000C0008482F538836E849208D90B00F552F3E1EF
:1000D0001200210E006E0006FEE11200849008005E
:1000E000F55201E10B008482F5CF83FF8492848274
:1000F000F538836E8492EDDF84800B00F552F3E1D6
:10010000120084908482EFCF83FF84928482EF3840
:10011000836E8492DEDF8480EC50F4E11200026A88
:1001200083502D6E0318030B0BE0033002E3E892BB
:1001300001D0E8822D18030B02E1020601D0022A49
:100140002DC003F012000490049283A602D004880C
:1001500001D0049804A604D004B802D01E0E056E87
:1001600004B807D0055204E104B402D0048004842A
:1001700001D0049404B607D004A805D0055201E0CC
:1001800004820494056A055201E0050604A802D021
:10019000048601D004961200C284C2B4FED7C4CF34
:1001A00007F0C450FF08086EC60E0F6E80A203D081
:1001B00008C013F002D007C013F001D8120008D80D
:1001C000116E133A05D8106E00EE0FF09ADF120090
:1001D00013500F0B090804E713500F0B370F03D010
:1001E00013500F0B3009120004A201D0807204A03A
:1001F00001D0807212000250010802E1062A04D0E8
:100200000250010F01E1060606A002D0808401D051
:10021000809406A202D0808601D08096120082903F
:10022000210E136E1AD807C013F017D8828082905F
:10023000220E136E12D808C013F00FD88280790EE8
:10024000C26E47DFC284C2B4FED7860E0F6EC4CF23
:1002500013F0B5DF610EC26E12009E9613C0C9FF87
:100260009EA6FED7C9CF14F01200410EC26EC18EF9
:1002700030DFC284C2B4FED7030E176EE80E186ECC
:10028000C3CF20F027EC04F0080E206E000E216E84
:100290004EEC03F019C013F004D8610EC26EC19E7B
:1002A000120000EE0BF0E86A13C017F00A0E206E81
:1002B00001EC04F01B503009ED6E17C013F0E9504B
:1002C0000908F1E100EE09F01CDF12008088010648
:1002D00003E1FA0E016E809812009EA4FED79E9450
:1002E0001200333228010C0600008051465056009F
:1002F000000001000180565501403433AB2A93249D
:100300000120721C9A1946175615B2134A1212117F
:100310000110100F390E7A0DCD0C310CA30B220BEE
:10032000AB0A3E0AD9097C092509D4088908430883
:100330000108C207880751071D07EC06BD06910694
:1003400067063F061906F505D205B1059105730547
:1003500056053A051F050605ED04D504BE04A8049C
:1003600093047E046A0457044504330422041104F0
:100370000104F103E103D303C403B603A9039C03FF
:100380008F03820376036A035F03540349033E032A
:1003900034032A03200316030D030403FB02F202B5
:1003A000E902E102D902D102C902C102BA02B202D3
:1003B000AB02A4029D0296029002890283027D0292
:1003C000770271026B0265025F025A0254024F0209
:1003D0004A0244023F023A02350231022C0227024D
:1003E00023021E021A02150211020D020902050261
:1003F0000102FD01F901F501F101ED01EA01E6015A
:10040000E201DF01DB01D801D501D101CE01CB0131
:10041000C801C401C101BE01BB01B801B501B301EE
:10042000B001AD01AA01A701A501A2019F019D0193
:100430009A0198019501930190018E018B01890128
:1004400087018401820180017E017B0179017701AE
:100450007501730171016F016D016B016901670124
:100460006501630161015F015D015B015901580193
:1004700056015401520151014F014D014B014A01F6
:100480004801470145014301420140013F013D014F
:100490003C013A01390137013601340133013101A0
:1004A00030012F012D012C012A01290128012601EB
:1004B000250124012201210120011F011D011C0130
:1004C0001B011A011901170116011501140113016D
:1004D000120110010F010E010D010C010B010A01A7
:1004E00009010801070106010501040103010201D8
:1004F0000101100E206008D020B6100C20B4200C92
:1005000020B2400C20B0800C20BC020C20BA040C9D
:1005100020B8080C1AC01EF01A6A19C01DF0196A1A
:1005200018C01CF0186A17C01BF0176A000C1B6A71
:10053000000C010E206497EF02F0D890F76A203487
:10054000F736F10FF66E020EF7220A0017C01CF004
:1005500018C01BF0F5501C02F4CF17F0F3CF18F0C1
:100560000900F5501B02F4CF19F01C02F3501926B4
:10057000F4501822E86A17220A00F5501B02F350C3
:100580001926F4501822E86A172220501802F3CFD7
:100590001AF0F4CF19F01702F35019261A501B5E07
:1005A00019501C5A1CAE000C1806E86A175A205045
:1005B0001B26000C17C02DF018C02EF019C02FF00C
:1005C00099EC02F017C02DF018C02EF02FC018F0D3
:1005D0001BC017F099EC02F018C019F02EC018F0EB
:1005E0002DC017F0000C206608D021C020F099EC37
:1005F00002F01BC01CF01B6A000C2050175CD8A036
:1006000090EF02F0D8A405D02150185CD8A090EF4C
:1006100002F017C02DF018C02EF018C027F017C038
:1006200018F0176A20C022F021C023F020BE1DD090
:100630002050E846F30FF66E020EF76AF722080024
:10064000F5502302F3CF21F0F4CF20F02202F35033
:100650002026F5502E02F3CF27F0F4CF18F02D020C
:10066000F3501826176AF45017229DEC02F0185028
:100670002102F350275CF4501B58D8A018061850DC
:100680002302F3502E5EF4502D5A18502202F350DC
:100690002D5E2DC01BF02EC01CF0000C1B6A1C6AC6
:1006A000E86A206608D021C020F0DAEC02F01BC016
:1006B0001CF01B6A000C17620CD018C017F019C090
:1006C00018F0F3EC02F018C019F017C018F0176A10
:1006D000000C19C01AF018C019F017C018F0176AEA
:1006E00017C02DF018C02EF019C02FF01AC030F02E
:1006F000020E166E010E296E20BE1CD079EC02F09F
:10070000296E21022050F3CF21F0F4CF20F02902EE
:10071000F350202629501A02F3CF30F0F4CF2FF0F7
:100720001802F3CF2EF0F4CF2DF01902F3502F263C
:10073000F4502E26D890F76A2034F736F10FF66E73
:10074000020EF7220A002DC017F02EC018F0A6ECFA
:1007500002F017A008D018682EC01BF020501B26EE
:10076000D8B0C8EF03F018502102F3502F5CF450BA
:100770001B58D8B00DD0180620501B26D8B008D072
:1007800018502102F3502F5CF4501B58D8A01806C3
:1007900018C02AF018502102F3502F5EF4502E5A40
:1007A00018502002F3502E5EF4502D5A2DAE05D075
:1007B0002A0621502F2620502E22164E09D02AC05C
:1007C0002BF02EC02DF02FC02EF030C02FF0BBD755
:1007D0002EC01BF02FC01CF0010E29640CD0294044
:1007E000206E79EC02F02F02F4CF1CF02E02F350B1
:1007F0001C26F4CF1BF0176A2AC019F02BC018F082
:10080000000C010E206497EF02F017C01BF020507F
:10081000176002D0176A000CD890F76AE836F736EE
:10082000F10FF66E020EF7220A00F5501B02F4CF0C
:1008300017F0F3CF18F00800F5501B02F4501826FB
:10084000E86A172220501702F3501B5E000C20505C
:100850001802F4CF18F0F3CF19F01702F4CF17F005
:0A086000F3501826E86A1722000C76
:020000040030CA
:08000000FFFAF6FEFFFFFBFF13
:00000001FF
